:0200000480007A
:100000009700000093808020F39F5030737012306F
:1000100097100000938000FF371111111301111187
:100020006F00A0001301000097100000938040FEB5
:10003000372122221301212217020000130212018C
:10004000670002001301000023A0200093804000FD
:100050003731333313013133170200001302020129
:10006000670012001301000023A0200093804000CD
:100070003741444413014144170200001302420176
:100080006700D2FF1301000023A0200093804000EE
:1000900097100000938080F8375155551301515542
:1000A0001702000013022201670002001301000082
:1000B00037616666130161661702000013023201A0
:1000C0006700020013010000377177771301717721
:1000D0001702000013020201670022001301000052
:1000E00037918888130181881702000013020201EA
:1000F000670032001301000097100000938000F5A4
:1001000093025000130360006387620037A199993E
:100110001301919913000000130000006385520041
:100120001301000097100000938000F39302500029
:10013000130360006397520037B1AAAA1301A1AA62
:10014000130000001300000063956200130100001B
:1001500097100000938000F1930250001303600099
:100160006347530037C1BBBB1301B1BB1300000091
:100170001300000063C56200130100009710000027
:10018000938000EF930250001303600063675300F5
:1001900037D1CCCC1301C1CC1300000013000000F8
:1001A00063E562001301000097100000938000EDEA
:1001B000930250001303600063D7620037E1DDDD76
:1001C0001301D1DD1300000013000000635553003C
:1001D0001301000097100000938000EB9302500081
:1001E0001303600063F7620037F1EEEE1301E1EEF6
:1001F000130000001300000063755300130100009A
:1002000073905F306F000003732F3034130FEFFFD4
:1002100073101F34732F3034137F3F0023A0E0018D
:10022000732F203423A2E00123A420009380C00078
:1002300073002030171500001305C5DC971500006A
:10024000938545E5370610F01306C6F26306B5023E
:100250008326C5002320D600832685002320D600D0
:10026000832645002320D600832605002320D600C0
:10027000130505016FF09FFD370510F0130505F21A
:040280002320050032
:10100000FFFFFFFFFFFFFFFFFFFFFFFFFFFFFFFFF0
:10101000FFFFFFFFFFFFFFFFFFFFFFFFFFFFFFFFE0
:10102000FFFFFFFFFFFFFFFFFFFFFFFFFFFFFFFFD0
:10103000FFFFFFFFFFFFFFFFFFFFFFFFFFFFFFFFC0
:10104000FFFFFFFFFFFFFFFFFFFFFFFFFFFFFFFFB0
:10105000FFFFFFFFFFFFFFFFFFFFFFFFFFFFFFFFA0
:10106000FFFFFFFFFFFFFFFFFFFFFFFFFFFFFFFF90
:10107000FFFFFFFFFFFFFFFFFFFFFFFFFFFFFFFF80
:10108000FFFFFFFFFFFFFFFFFFFFFFFFFFFFFFFF70
:040000058000000077
:00000001FF
